:100000001D308A00102D0000FF00030E8301A100A7
:100010000A08A0008A010408A2007708A300780853
:10002000A4007908A5007A08A6007B08A70083131E
:1000300083120B1E1D288B1842288C308400801ED2
:1000400023288C1A45288C308400001C29280C1881
:1000500048288C308400801C2F288C184B282208BC
:1000600084002308F7002408F8002508F900260872
:10007000FA002708FB0020088A00210E8300FF0EEB
:100080007F0E09008A110A123E2B8A110A12002DD6
:100090008A110A1278298A110A12C22B0A108A10B0
:1000A0000A1182070D340A344B342D344A34753426
:1000B0006E3469346F34723420344F3470346534A4
:1000C00072346134743469346E3467342034533498
:1000D00079347334743465346D340D340A34003437
:1000E0000A108A100A1182076B344A344F34533491
:1000F0002034253473342D34253430343234643490
:10010000203428342534733429342C3420344B34AF
:100110002D345434653461346D34203453344134D7
:100120000D340A3400340A108A100A11820741344F
:1001300000340A108A100A11820735343134303401
:100140002E34303430343134383400340A108A10CC
:100150000A11820745342D344D34613469346C34CE
:1001600020343A34203469346E3466346F34403489
:100170006B342D347434653461346D342E3463340F
:100180006F346D340D340A3400340A108A100A11A9
:10019000820755346E346B346E346F3477346E347A
:1001A000203443346F346D346D3461346E346434D0
:1001B00020343F3421340D340A3400340A108A10BC
:1001C0000A1182075334453454340A3400340A1077
:1001D0008A100A118207533445344C344534433471
:1001E0005434203430340A3400340A108A100A118E
:1001F000FC3E03188A0A820049346E347434653434
:1002000072346E3461346C34203462346534683452
:100210006134763469346F34723420347334743416
:1002200061347234743469346E3467340D340A3492
:1002300000340A148A100A1182074E346F342034B5
:100240007434613473346B34203461346C346F34FF
:10025000753465346434203466346F347234203439
:1002600074346834693473342034733465347434CA
:10027000743469346E3467342C34203472347534F9
:100280006E3420346134733420346434653466341D
:10029000613475346C34743420346D346F346434A8
:1002A00065340D340A340034831603171E080739E9
:1002B000F7001E0CF800F80CF80C1F30F805780851
:1002C00020078400831321188317F801F80AF70A1E
:1002D0006A29F80DF70B69299F0803197229780814
:1002E00080047529F8097808800583120313003407
:1002F000FE308F003D308E00C70A4708033C0318CC
:10030000AC29C7010130C3070318C40A0319C50A81
:100310000319C60AC80803199729C90A4908633C82
:1003200003189729C901C80B9729AB01AA01F0014D
:10033000051EF00A0030891C0130F7000310F70D8C
:100340007708F0040030091D0130F700F70DF70DB4
:10035000FC30F7057708F004AA08031DB22907113D
:100360008810D429AA1BC4292A08003C0318C429D0
:10037000AA1BBE292A082C02031CC12907118810B8
:10038000C32907158810D429AA1FD4292A08003C9C
:10039000F700F71BCF2977082C02031CD22907117D
:1003A0008810D42907118814AB08031DDA29871097
:1003B0000810FC29AB1BEC292B08003C0318EC2986
:1003C000AB1BE6292B082C02031CE9298710081017
:1003D000EB2987140810FC29AB1FFC292B08003CD3
:1003E000F700F71BF72977082C02031CFA2987105E
:1003F0000810FC2987100814AC0A2C08133C0318B9
:10040000022AAC01F408031D072A0812132AF50A70
:100410007408643C7502031C132A081E112A081272
:10042000122A0816F501F10803196A2A7208F70062
:100430007308FA007A08031D202AF7080319412AD5
:1004400001307A02031D282AF43077020319462A64
:1004500003307A02031D302AE830770203194B2A51
:1004600005307A02031D382ADC3077020319502A3E
:1004700007307A02031D402AD03077020319552A2B
:100480005A2A711A8613711888165A2A71188812F6
:10049000F11808175A2AF1180813711988175A2ADF
:1004A00071198813F11906175A2AF1190613711ACE
:1004B00086175A2AF20A0319F30A7308083C03182C
:1004C0006A2AFF3A031D682A7208C23C03186A2A86
:1004D000F301F2012D186E2AC21D182B630B922A0C
:1004E0000310620D4A3E840083139F18752A1E086C
:1004F000FA0083161E088000840A7A08800064309F
:1005000083126207840083130008831603179D007B
:100510009E0001309F00A101A0018312031354210A
:10052000E30A182B6308033C031D162B0310620D0E
:10053000103E840083179F189B2A1E08FA0083161A
:100540001E088000840A7A08800003108312620D5E
:10055000103EF8000130FA000318FA0A78088316F2
:1005600003179D007A089E00031083120313620D87
:100570004A3E84008313840A000883160317A000F0
:10058000840300089F00031083120313620D103EC2
:1005900084008317840A0008FA0084030008831685
:1005A00003179F027A08031C7A0FA0022008FA00A2
:1005B0001F08A01FE42A1F08003CF700FA012008CA
:1005C000031C200FFA0277089F007A08A0001D087C
:1005D000840083131E188317840A20088000840374
:1005E0001F088000643083120313620784008313A2
:1005F0000008831603179D009E009F01A101A00122
:10060000831203135421E20A62080B3C03180B2BDC
:10061000E201AD16C211620DF700F70DFC30F705CF
:100620001F08C33977049F00E301182B9F14E30AC6
:100630000F08FA000E08F7000F087A02031D182BA6
:100640007708831603179B007A089C001C08FE3C61
:10065000031C382B031D302B1B083C3C031C382B80
:10066000FF30831203138F00DC308E0083160317D4
:10067000831203130C108A110A122F28AD1C572B5A
:10068000BF012F303F07840083130030061C013068
:1006900080000B121030F80005389200BE3083162F
:1006A00092008312910183168C14831242148B10D2
:1006B0008A110A122F2801303E02EF3E03188E2BBA
:1006C000113E912B0530AA001430AB008E2B0A305E
:1006D000AA00AB008E2B1430AA000530AB008E2B85
:1006E000F630AA000A30AB008E2BAA01AB018E2B8C
:1006F0000A30AA00F630AB008E2BFB30AA00EC309B
:10070000AB008E2BF630AA00AB008E2BEC30AA008B
:10071000FB30AB008E2B8E2B8E2B8E2B8A110A1268
:10072000432C0A148A140A118207622B672B6B2B45
:10073000702B752B782B7D2B822B862B8E2B8E2B63
:100740008B2B8E2B8E2B8E2B8C2B8D2B83160317A6
:100750009C019C011C081F3C031CBF2B831203132C
:1007600086160830F700F70BB32B00008612053011
:10077000F700F70BB92B831603179C0AAA2B8312D9
:1007800003130034831603171B1083120313421C38
:10079000512C91012030F80005389200AC308316BE
:1007A00092008312BF0A3F080D3C031CE02B2F3040
:1007B0003F07840083130030061801308000502C5E
:1007C0002F0B432C300B432C320E831603179C0047
:1007D000F0309C0583120313330DF700F70DF70D6E
:1007E000F830F7057708831603179C048312031368
:1007F000340DF700F70DFC30F70577088316031763
:100800009C04031083120313350D831603171C0475
:10081000831203133604BD00370E831603179C00A2
:100820009C0DE0309C0583120313380EF700F03066
:10083000F7057708831603179C0483120313390DF9
:10084000F700F70DF70DF830F70577088316031753
:100850009C04831203133A0DF700F70DFC30F705E3
:100860007708831603179C040310831203133B0DB0
:10087000831603171C04831203133C04BE00AD1738
:10088000AD1D432C5B2B0B1683168C101830F80013
:1008900083129200AC308316920083128B104210A8
:1008A000FC2CC21CF02C0830F80005389200C8302F
:1008B000831692008312421191013F08023C031CEF
:1008C000672C831603171B14C12C831203133F08D4
:1008D0000D3C0318842CC2100B1683168C100830A4
:1008E000F80083129200D7308316920005308312ED
:1008F000900083160C1483128B102D13831603178C
:100900001B14C12C831203133F08083C0318A82CA6
:100910003F080D3C031CA82C08303F02F800203093
:10092000F700F8080319982C0310F70CF80B942C17
:10093000770840050319A22C831603171B14A52C56
:1009400083120313831603171B10C12C8312031386
:1009500003303F02F8001030F700F8080319B42CF8
:100960000310F70CF80BB02C770841050319BE2CC7
:10097000831603171B14C12C83120313831603174A
:100980001B10831203132D1BD42C831603171B1C5F
:10099000CC2C83120313D42C83120313A6232D1300
:1009A000BF0A91018C10ED2C2D1FE62C8316031726
:1009B0001B18DD2C83120313E62C83120313A623CA
:1009C000BF0A2D13421591018C10ED2C00302D1B08
:1009D0000130BF074030AD06861242195B2CFC2C5B
:1009E0000B1683168C101830F80083129200AC306E
:1009F0008316920083128B108C108A110A122F28F2
:100A00008C1E332D2D1E102DF608031D102D8C1E4F
:100A1000072D1A08831603179B00302D831203132A
:100A2000A0302E07840083138C1E142D1A0880001A
:100A3000A0302E078400831300080D3C0319282DD5
:100A4000A0302E078400831300080A3C031D292DC3
:100A50002D162E084E3C031C2E2DAE0A83160317AE
:100A600083120313002D8C128A110A122F280317E8
:100A70004008F8013F020318402D3F08F7004C2DB5
:100A8000F7010830C100BF0DF70D400877020318C9
:100A9000F700F80DC10B432D03130034203003176A
:100AA0003A1E3030BB003908F700B91F5E2DF70938
:100AB000F70A7708B9002D30BB00BA173908BF0014
:100AC0006430C0000313372577080317B9003030AE
:100AD0007807BC003908BF000A30C000031337256F
:100AE000303077070317BE0030307807BD003B0871
:100AF000F700BA1D7D2DBA1F3A113A1A8A2DBA1F76
:100B0000A52D3A19A52D7708BC00BA18A52D770890
:100B1000BD00A52D30303C02031DA52D7708BC007B
:100B20002030BB00BA1D982D3A11BA14BA1FBA1062
:100B300030303D02031DA52D7708BD002030BC00DC
:100B4000BA1D982DBA10BA1F3A103A1DAD2D3B08A8
:100B500003130C1EA92D99000317BA1CB52D3C08D0
:100B600003130C1EB12D990003173A1CBD2D3D082F
:100B700003130C1EB92D990003173E0803130C1E16
:100B8000BF2D990000340317B8013F3083160313BB
:100B900085001F30860098308700003088000914D7
:100BA000891409158312850186018701880189014D
:100BB0001F179F1783169F1783121F1471308316F8
:100BC0008F000F0883120317B8013808093C031C73
:100BD000FD2D0310380D4A3E84008313840A8001E2
:100BE000840380010310380D103E84008317840AAB
:100BF000800184038001B80AE52D0313AA01AB012B
:100C00008513081188112F30E4004230E5002F30A1
:100C1000E6004330E7002F30E8004330E90042307F
:100C2000ED004330EE004230EC004330EF003D3049
:100C3000EA00EB000317B901390803134E2003172C
:100C4000B90AF70003130C1E232E99001D30031759
:100C50003902031D1C2EB901390803137020031734
:100C6000B90AF70003130C1E332E99000530031741
:100C70003902031D2C2EB9013908031393200038C3
:100C800003194B2E0317B90A03130C1E452E9900A6
:100C900003173C2E03132D300C1E4C2E99000930E7
:100CA0000317B9000130BA0003134E2520300C1E83
:100CB000572E990028300C1E5B2E99000317B9019E
:100CC000390803139920003803196F2E0317B90A46
:100CD00003130C1E692E99000317602E03131030A6
:100CE0000317B9003908031370200317B90AF70076
:100CF00003130C1E792E99001E3003173902031DB1
:100D0000722EB90139080313A6200317B90AF70098
:100D100003130C1E892E99001A3003173902031D84
:100D2000822E03131F179F1783169F1783121F14FA
:100D3000831603170908C0390F38890003131F12DF
:100D40009F123F30031788000030F800831203130E
:100D50001F08C33978049F00FE308F003D308E009D
:100D60000530900083160C1483122D1DBA2E8316A5
:100D70008C1683128316011383120B16C0308B045A
:100D8000F001051EF00A0030891C0130F700031045
:100D9000F70D7708F0040030091D0130F700F70D5A
:100DA000F70DFC30F7057708F00491011030F800DA
:100DB00005389200AC308316920083128A150A1609
:100DC000902D2D100317641CE82E03132D14031708
:100DD00003130034AD100317641CF12E0313AD147C
:100DE0000317031300342D110317641CFA2E031389
:100DF0002D15031703130034AD110317641C032FC3
:100E00000313AD15031703130034AD120034C215DC
:100E1000AD12003410300317EC00F701FA01E90CB1
:100E2000E80C031C192F6A08F7070318FA0A6B0865
:100E3000FA07FA0CF70CF90CF80CEC0B0F2F031354
:100E40000034031767086B068039831695008312F8
:100E5000E71F352FE409E509E609E709E40A031964
:100E6000E50A0319E60A0319E70AEB1F422FE8090E
:100E7000E909EA09EB09E80A0319E90A0319EA0A88
:100E80000319EB0AF701F801F901FA018316900141
:100E900091019201930183126B086A04690468044A
:100EA00003199E2F20308316940003108312E40D43
:100EB000E50DE60DE70D8316900D910D920D930D46
:100EC00083126B0883161302031D762F83126A08A0
:100ED00083161202031D762F8312690883161102EE
:100EE000031D762F8312680883161002031C972FA8
:100EF000831268088316900283126908031C690F25
:100F0000822F852F8316910283126A08031C6A0FB1
:100F10008A2F8D2F8316920283126B08031C6B0F8E
:100F2000922F952F83169302831203148316F70DC5
:100F3000F80DF90DFA0D940B552F83128316951F9A
:100F4000AC2FF709F809F909FA09F70A0319F80AA1
:100F50000319F90A0319FA0A9030840083178312DF
:100F600003130034031767080313AA000317680864
:100F70000313AB00AA1BC32F2A08143C0318C32F6A
:100F80001430AA00CA2F2A08803A6B3C031CCA2FCF
:100F9000EC30AA00AB1BD32F2B08143C0318D32F23
:100FA0001430AB00DA2F2B08803A6B3C031CDA2F8D
:100FB000EC30AB000034683084008317000803195C
:100FC000EE2F0230F800F701F70BE42FF80BE32FB8
:100FD0009730F700F70BEA2F800BE12F0034141342
:100FE000831691159119F22F77189112771C91168B
:0E0FF0001116111AF92F83121308F80000349D
:101000000317E401E501A31F0828A71F14280A28D5
:10101000A71B1B2823082702031C1B28031D1428B9
:101020002608220203181B282308E5002208E400F2
:101030000930E60021282708E5002608E4000B30E7
:10104000E600A51B2D2825086502031C3328031D77
:101050002D2864082402031833282508E5002408F5
:10106000E4000A30E600A11B3F2821086502031CAA
:101070004528031D3F28640820020318452821083D
:10108000E5002008E4000830E60008306602FC3E77
:1010900003181E29043E03132129FB300317E70020
:1010A000E8008A110313B2278A15FF300317E800FE
:1010B0008A110313DB278A1505300317E700FC307C
:1010C000E8008A110313B2278A1502300317E700DC
:1010D000AF30E8008A110313DB278A150317E70BEB
:1010E00068280A30E700E8008A110313B2278A153E
:1010F00032300317E8008A110313DB278A15031720
:101100001E29FB300317E700E8008A110313B227FA
:101110008A15FF300317E8008A110313DB278A15AD
:10112000FC300317E7000530E8008A110313B227EB
:101130008A1502300317E700AF30E8008A11031365
:10114000DB278A150317E70B9C280A30E700E80025
:101150008A110313B2278A1532300317E8008A1167
:101160000313DB278A1503171E29FB300317E7003B
:10117000E8008A110313B2278A15FF300317E8002D
:101180008A110313DB278A1505300317E700FC30AB
:10119000E8008A110313B2278A1504300317E70009
:1011A000AF30E8008A110313DB278A150317E70B1A
:1011B000D0280A30E700E8008A110313B2278A1505
:1011C00032300317E8008A110313DB278A1503174F
:1011D0001E29FB300317E700E8008A110313B2272A
:1011E0008A15FF300317E8008A110313DB278A15DD
:1011F000FC300317E7000530E8008A110313B2271B
:101200008A1504300317E700AF30E8008A11031392
:10121000DB278A150317E70B04290A30E700E800EB
:101220008A110313B2278A1532300317E8008A1196
:101230000313DB278A1503171E2903170313421212
:1012400000340A148A100A118207E9284D28B528AB
:1012500081280317B80138088A110313F5208A156D
:101260000317B80AF70003130C1E342999001C3029
:1012700003173802031D2B297008013A03130319C1
:101280004829033A0319FC2C013A0319692DAD2DA5
:101290000317CE01CF01D001D1010F30D200D3010D
:1012A000BC30D4000230D500BC30D6000230D700AC
:1012B000BC30D8000230D900BC30DA000230DB008C
:1012C000DC01DD01DE01DF01E001E101E201E3011A
:1012D000E4018A110313E1268A150317E4018A1138
:1012E0000313EA268A150317E4018A110313F32670
:1012F0008A150317E4018A110313FC268A158A1143
:1013000005278A158A1107278A15AD1E8529031717
:10131000BB01BA01B901B801BF01BE01BD01BC01E9
:10132000C0014008053C031C092A0310400D103E73
:1013300084008317840A0008E50084030008E400A1
:10134000E51BB9296508013C0318B929FF3A031DBB
:10135000AD296408BC3C0318B9290310400D423E76
:1013600084008317840A0130800084035E3080008B
:10137000072A0310400D103E84008317840A0008DA
:10138000E50084030008E400E51BCD29E508031D02
:10139000D7296408C73C031CD7290310400D423EDF
:1013A00084008317840A800184038001072A0310C4
:1013B000400D423EF8000130FA000318FA0A78089E
:1013C000E4007A08E5000310400D103E8400831706
:1013D000840A0008E70084030008E600C830E6023B
:1013E0000030031C0130E7020310670CFA00660CA2
:1013F000F900E6007A08E7006408840083136518A2
:101400008317840A67088000840366088000C00A86
:101410009129C0014008053C031C8A2A2C30400752
:1014200084008317E5010008E400E41BE5030310D2
:10143000400D423E84008317840A0008FA008403AA
:101440000008E6007A08E7006508E9006408E8009B
:101450006708EB006608EA008A1103130A278A1559
:101460007908FA007808F7007908F800F901FA011C
:10147000F81F3C2AF903FA0377080317B80778081E
:101480000318780FB90779080318790FBA077A0893
:1014900003187A0FBB073230400784008317E50139
:1014A0000008E400E41BE5030310400D423E840005
:1014B0008317840A0008FA0084030008E6007A080B
:1014C000E7006508E9006408E8006708EB006608C3
:1014D000EA008A1103130A278A157908FA007808A6
:1014E000F7007908F800F901FA01F81F792AF903E1
:1014F000FA0377080317BC0778080318780FBD07AD
:1015000079080318790FBE077A0803187A0FBF0706
:10151000C00A0A2A3B08E7003A08E6003908E50055
:101520003808E400EB01EA01E9016430E8008A11BF
:10153000031321278A157A080317E7007908E600C4
:101540007808E5007708E40005306407B80065080E
:10155000B900003003180130B9076608BA0000303E
:1015600003180130BA076708BB00003003180130C8
:10157000BB073F08E7003E08E6003D08E5003C08E1
:10158000E400EB01EA01E9016430E8008A11031389
:1015900021278A157A080317E7007908E6007808FA
:1015A000E5007708E40005306407BC006508BD006D
:1015B000003003180130BD076608BE000030031874
:1015C0000130BE076708BF00003003180130BF07B5
:1015D000BB1B0B2BBB08031DF72ABA08031DF72AF8
:1015E000B908031DF72A3808003C03180B2BBB1B56
:1015F000062BBB08031D0B2BBA08031D0B2BB908C8
:10160000031D0B2B3808043C031C0B2BBB01BA0138
:10161000B9010530B800BB1F2E2BBB1F282B3B0880
:10162000FE3C03182E2BFF3A031D282B3A08FE3CE4
:1016300003182E2BFF3A031D282B3908FE3C0318F4
:101640002E2BFF3A031D282B3808FB3C03182E2BAA
:10165000FF30BB00BA00B900FB30B800BF1B512BF4
:10166000BF08031D3D2BBE08031D3D2BBD08031DF8
:101670003D2B3C08003C0318512BBF1B4C2BBF08D3
:10168000031D512BBE08031D512BBD08031D512BFB
:101690003C08043C031C512BBF01BE01BD010530B9
:1016A000BC00BF1F742BBF1F6E2B3F08FE3C0318EE
:1016B000742BFF3A031D6E2B3E08FE3C0318742B5F
:1016C000FF3A031D6E2B3D08FE3C0318742BFF3AB6
:1016D000031D6E2B3C08FB3C0318742BFF30BF002E
:1016E000BE00BD00FB30BC00C101A31B822B230840
:1016F000003C0318822BFF3A031D812B22082B3C50
:10170000031CC10AA51B8F2B2508003C03188F2B37
:10171000FF3A031D8E2B24082B3C031CC10AA11B7E
:101720009C2B2108003C03189C2BFF3A031D9B2B8C
:1017300020082B3C031CC10AA71BA92B2708003C2F
:101740000318A92BFF3A031DA82B26082B3C031CCA
:10175000C10A4108013C031CB92BBF01BE01BD01F8
:10176000BC01BB01BA01B901B80103134212F12C4B
:1017700003174108043C031DEF2C56085407E400EE
:101780005508E50057080318570FE5075808E40700
:1017900059080318590FE5075A08E4075B080318AE
:1017A0005B0FE507650CCF00640CCE00CF0CCE0CB0
:1017B0003F30CF05D3015030D200CF08031DE72BB7
:1017C0004E08633C031CE72BD3011430D2002408DD
:1017D0002207E4002308E50025080318250FE50784
:1017E0002008E40721080318210FE5072608E4076D
:1017F00027080318270FE5076508E7006408E600D7
:10180000E9010430E800670869068039EB00E71F4A
:101810000E2CE609E709E60A0319E70AE91F152C69
:10182000E809E909E80A0319E90AF801F901F701E9
:10183000FA016908031D1F2C68080319392C1030A0
:10184000EA000310E60DE70DF70DFA0D69087A02BC
:10185000031D2C2C68087702031C352C6808F7023E
:10186000031CFA036908FA020314F80DF90DEA0BD8
:10187000212CEB1F402CF809F909F80A0319F90A81
:101880007808D0007908D1001E305007E4005108D4
:10189000E5000318E50A65084F02031C552C031DDB
:1018A000682C4E086402031C682C1E305002E400B1
:1018B0005108E5000030031C0130E5024F086502C5
:1018C000031C6B2C031D682C64084E0203186B2C40
:1018D0000313421203170313421A912C03175508DE
:1018E000DD005408DC005708DF005608DE00590808
:1018F000E1005808E0005B08E3005A08E200230812
:10190000D5002208D4002508D7002408D6002108D5
:10191000D9002008D8002708DB002608DA000313C6
:101920004216031752085407F8005508FA005308E6
:101930000318530FFA077808A31BA82C7A08230270
:10194000031CA82C031DEA2C22087802031CEA2C95
:1019500052085607F8005708FA0053080318530FA7
:10196000FA077808A51BBE2C7A082502031CBE2C9A
:10197000031DEA2C24087802031CEA2C520858079D
:10198000F8005908FA0053080318530FFA077808AB
:10199000A11BD42C7A082102031CD42C031DEA2C91
:1019A00020087802031CEA2C52085A07F8005B084A
:1019B000FA0053080318530FFA077808A71BEE2CF8
:1019C0007A082702031CEE2C031DEA2C2608780255
:1019D0000318EE2C03130020ED2C0317F22C031335
:1019E000002003173808E7003C08E8008A110313B9
:1019F000B2278A157F29C12D0317E4018A11031329
:101A0000E1268A150317E4018A110313EA268A15D1
:101A10000317E4018A110313F3268A150317E4015F
:101A20008A110313FC268A1505300317E700E80026
:101A30008A110313B2278A158A1105278A158A117C
:101A400007278A15AD1E222D0317A11B312D210852
:101A5000023C031C462D031D312D2008BC3C031CF9
:101A6000462DA51B3D2D2508023C031C462D031DBC
:101A70003D2D2408BC3C031C462D0530E700E80042
:101A80008A110313B2278A15672D0317A11F4B2D47
:101A9000A51F572D4D2DA51B602D21082502031CC8
:101AA000602D031D572D240820020318602D0A30D5
:101AB000E700E8018A110313B2278A15672D03177F
:101AC000E7010A30E8008A110313B2278A151C2D9A
:101AD000C12D0317E4018A110313E1268A150317A8
:101AE000E4018A110313EA268A150317E4018A1117
:101AF0000313F3268A150317E4018A110313FC2646
:101B00008A1508300317E7000430E8008A11031330
:101B1000B2278A1504300317B800AF30E8008A11E5
:101B20000313DB278A150317B80B8D2DFC30E70054
:101B3000F830E8008A110313B2278A15043003171E
:101B4000B800AF30E8008A110313DB278A150317AA
:101B5000B80BA12D0313812DC12D0317B80138082F
:101B60008A11031319218A150317B80AF700031302
:101B70000C1EB82D9900363003173802031DAF2D07
:101B800003138A150A16972D0317C501C3010A30DE
:101B9000C400C20140084104031DD12D0030F800EB
:101BA000C42E4508C50A40078400831341188317D3
:101BB0000008C60046082D3C031DEA2D0130C30075
:101BC0004508C50A4007840083134118831700089D
:101BD000C600F72D46082B3C031DF72D4508C50A06
:101BE000400784008313411883170008C600460885
:101BF0002F3C0318BA2E4608393C031CBA2E46085F
:101C0000303C031D232E45084007840083134118F0
:101C100083170008783C0319172E450840078400F5
:101C20008313411883170008583C031D232E1030DE
:101C3000C400C50A4508C50A40078400831341183B
:101C400083170008C60044080A3C031D682E460896
:101C50002F3C0318672E4608393C031C672E0A30B8
:101C6000C7004208C800F701F801470803104818E8
:101C7000F707F70CF80CC818F707F70CF80C481919
:101C8000F707F70CF80CC819F707F70CF80C481A07
:101C9000F707F70CF80CC81AF707F70CF80C481BF5
:101CA000F707F70CF80CC81BF707F70CF80C7808C7
:101CB000C700303046024707C2004508C50A400742
:101CC00084008313411883170008C600272EBA2EFC
:101CD0004408103C031DBA2E4608603C0318772EBA
:101CE00046087A3C031C772E4608DF39782E4608D2
:101CF000C60046082F3C0318812E4608393C0318BD
:101D0000892E4608403C0318BA2E4608463C031C60
:101D1000BA2E46082F3C03189A2E4608393C031C5D
:101D20009A2E420EC700F030C705303046024707F2
:101D3000C200A32E420EC700F030C7054130460254
:101D40000A3E4707C2004508C50A400784008313BE
:101D5000411883170008C6004608603C0318B72ED8
:101D600046087A3C031CB72E4608DF39B82E4608D1
:101D7000C600792E430BC22E44080A3C031DC22E16
:101D8000C209C20A4208F8000313003462300C1E74
:101D9000C72E99002C300C1ECB2E99000317B801CA
:101DA00038088A11031393208A1500380319E12E8D
:101DB0000317B80A03130C1EDB2E99000317D02E4D
:101DC00003132D300C1EE22E990009300317B900C1
:101DD0000130BA008A1103134E258A150D300C1EEE
:101DE000EF2E99000A300C1EF32E99008A150A1660
:101DF0000B2D02300317BD00BE01A0303D0784004B
:101E0000831300082C3C0319302FA0303D078400B9
:101E1000831300080A3C0319302FA0303D078400CB
:101E2000831300080D3C0319302F38303E07F800AB
:101E30000130FA000318FA0A7808C0007A08C100D5
:101E4000A0303D07840083130008C20040088400CE
:101E500083134118831742088000BD0ABE0AFD2E75
:101E600038303E078400831780010130C1003830CC
:101E7000C0000313C42578080317BF00A0303D0736
:101E80008400831300080A3C03194E2FA0303D073D
:101E90008400831300080D3C031D612FC00140081E
:101EA0008A110313C5208A150317C00AF70003130C
:101EB0000C1E582F9900143003174002031D4F2F9A
:101EC000CC2FBD0ABE01A0303D078400831300085B
:101ED0000A3C03198E2FA0303D07840083130008AD
:101EE0000D3C03198E2F38303E07F8000130FA0000
:101EF0000318FA0A7808C0007A08C100A0303D072C
:101F0000840083130008C200400884008313411832
:101F1000831742088000BD0ABE0A632F38303E078F
:101F20008400831780013F080313AA00AA1B9F2F78
:101F30002A08143C03189F2F1430AA00A62F2A0841
:101F4000803A6B3C031CA62FEC30AA00013003172B
:101F5000C1003830C0000313C4257808AB00AB1BA8
:101F6000B82F2B08143C0318B82F1430AB00BF2F28
:101F70002B08803A6B3C031CBF2FEC30AB00643065
:101F80000C1EC02F99000D300C1EC42F99000A3072
:101F90000C1EC82F9900031703138A150A160B2D60
:101FA00065300C1ED12F99002C300C1ED52F9900B6
:101FB0002A080317B9001F30BA008A1103134E25EF
:101FC0008A152C300C1EE22F99002B080317B9003C
:101FD0001F30BA008A1103134E258A150D300C1ECE
:101FE000EF2F99000A300C1EF32F99008A150A165C
:021FF0000B2DB7
:1020000002300317BD00BE01A0303D0784008313DA
:1020100000082C3C03193328A0303D0784008313AB
:1020200000080A3C03193328A0303D0784008313BD
:1020300000080D3C0319332838303E07C00001303A
:10204000C1000318C10AA0303D07840083130008B3
:10205000C20040088400831341188317420880009F
:10206000BD0ABE0A042838303E0784008317800169
:102070000130C1003830C0000A128A150313C4258C
:102080000A168A1178080317BF00A0303D078400A4
:10209000831300080A3C03195528A0303D0784002B
:1020A000831300080D3C031D6828C00140080A1274
:1020B0000313C5200A160317C00AF70003130C1EEA
:1020C0005F289900143003174002031D56283B294E
:1020D000BD0ABE01A0303D078400831300082C3CDC
:1020E00003199928A0303D078400831300080A3C97
:1020F00003199928A0303D078400831300080D3C84
:102100000319992838303E07C0000130C100031878
:10211000C10AA0303D07840083130008C2004008B4
:10212000840083134118831742088000BD0ABE0A49
:102130006A2838303E07840083178001A0303D07AD
:102140008400831300080A3C0319AE28A0303D0721
:102150008400831300080D3C031DC128C001400802
:102160000A120313C5200A160317C00AF700031347
:102170000C1EB8289900143003174002031DAF2825
:102180003B293F080313AA0001300317C100383070
:10219000C0000A128A150313C4250A168A1178088A
:1021A000AB000317BD0ABE01A0303D0784008313B6
:1021B00000080A3C0319FB28A0303D078400831364
:1021C00000080D3C0319FB2838303E07C0000130E1
:1021D000C1000318C10AA0303D0784008313000822
:1021E000C20040088400831341188317420880000E
:1021F000BD0ABE0AD42838303E0784008317800108
:102200000313AA1B0A292A08143C03180A291430AC
:10221000AA0011292A08803A6B3C031C1129EC30D2
:10222000AA00AB1B1A292B08143C03181A291430D6
:10223000AB0021292B08803A6B3C031C2129EC3090
:10224000AB0001300317C1003830C0000A128A15F4
:102250000313C4250A168A117808C80061300C1EC1
:102260002F2999000D300C1E332999000A300C1EBD
:1022700037299900031703138A150A160B2DF70146
:10228000F801F901FA010317CC01CD01CE01CF010C
:102290004B084A044904480403197E292030D00021
:1022A0000310C40DC50DC60DC70DCC0DCD0DCE0D43
:1022B000CF0D4B084F02031D67294A084E02031D2C
:1022C000672949084D02031D672948084C02031C71
:1022D00078294808CC024908031C490FCD024A0856
:1022E000031C4A0FCE024B08031C4B0FCF020314F2
:1022F000F70DF80DF90DFA0DD00B50294C30840074
:1023000083170313003402300317BD00BE01A03051
:102310003D078400831300080A3C0319B229A0304A
:102320003D078400831300080D3C0319B22938309F
:102330003E07F8000130FA000318FA0A7808BF00D7
:102340007A08C000A0303D07840083130008C10054
:102350003F08840083134018831741088000BD0A9A
:10236000BE0A872938303E07840083178001013078
:10237000C1003830C0000A128A150313C4250A169A
:102380008A117808F4007408643C0318C929643081
:10239000F40068300C1ECA2999000D300C1ECE299D
:1023A00099000A300C1ED22999008A150A160B2DA5
:1023B0000317BC1BEE290F30F7003B0EF7050A3060
:1023C00077020318E6293030F707E8293C08F707B9
:1023D000770803130C1EEA29990003170F30BB0579
:1023E0000A303B020318F6293030F829BC133C08A8
:1023F000BB073B0803130C1EFB2999000034941300
:102400008C118316031711088312031393000230F3
:10241000941B112A8C1D0A2A00308316111B0130CF
:102420008312F80000346A300C1E142A990003301D
:102430000317B8003808FD3C031C692A83160313F0
:1024400011141118212A0130831203173802BA001F
:102450008316910083120313FF21F808031D602ADD
:1024600083160317910183120313FF21831691141E
:102470009118382A831203173808831691008312A3
:102480000313FF21F7010A12EF270A167808031732
:10249000B90083160313111511194C2A0130831248
:1024A00003173802BA002C3003130C1E552A99006A
:1024B00003173A08BB005730BC000313D821652A24
:1024C000831611151119622A831202300317B807F7
:1024D0001A2A0D3003130C1E6B2A99000A300C1EA9
:1024E0006F2A99008A150A160B2D03173908073928
:1024F000F700390CF800F80CF80C1F30F8057808D4
:102500003A07840083133B1883170008F800F70A82
:102510008A2AF80CF70B892A03138A110A16ED2A66
:1025200083162208303A83120319A32A013A0319A9
:10253000A72A033A0319AB2A013A0319AF2A073A2B
:102540000319B32AB82A45300317B800CC2A4630FD
:102550000317B800CC2A47300317B800CC2A36300E
:102560000317B800CC2A37300317B800CC2A03135E
:102570000317B90139080A120313C5200A160317F5
:10258000B90AF70003130C1EC32A9900143003176D
:102590003902031DBA2ACC2A831603132408333CBC
:1025A000031DE12A30302202F8000130F700F8085C
:1025B0000319DE2A0310F70DF80BDA2A7708F10465
:1025C000542B2408323C031D172B831203173808A1
:1025D000B900BB01BA010313752A781C022BA801AC
:1025E0008B1BA8178B130317380883169E009F01B7
:1025F000A101A0010A128312031354210A16A81B79
:102600008B17152BA8018B1BA8178B1303173808E2
:1026100083169E0001309F00A101A0010A128312BF
:10262000031354210A16A81B8B17442B8316240866
:10263000303C031D302B8312A8018B1BA8178B1372
:102640000317380883169E009F01A101A0010A12FA
:102650008312031354210A16A81B8B17442B8316CD
:102660008312A8018B1BA8178B1303173808831636
:102670009E0001309F00A101A0010A1283120313E2
:1026800054210A16A81B8B17303083162202F8003B
:102690000130F700F8080319512B0310F70DF80B60
:1026A0004D2B7708FF3CF1056C3083120C1E562B26
:1026B00099000D300C1E5A2B99000A300C1E5E2B0F
:1026C00099008A150A160B2D0317C0010408BF00D4
:1026D0004010831B4014B91F752BBF173F1EBF0A44
:1026E000B809B909B80A0319B90A390EF038BB009C
:1026F000BB07E23EBC00323EBE0039080F39BC07C2
:10270000BC07BE07E93EBD00BD07BD07380E0F3947
:10271000BD07BE07BD0DBE0DBE09BE0D38080F3981
:10272000BE07BB0D0730BA000A30BE07BD03031C4D
:10273000952BBD07BC03031C992BBC07BB03031CD3
:102740009D2BBB07BA03031CA12B3A3084008317CF
:1027500007303F053F1384033F05031DB62B3F1A87
:10276000840A3F1AB62B2030F700D32B84073E3063
:10277000040203193F170008F700031DC72B3F1B76
:10278000C72B3F1AD92BBF19C72B2030D22BBF1F05
:10279000CF2B2D30F70084033F13BF13D32BBF156E
:1027A0003F123030F707770803130C1ED52B990022
:1027B0000317840A3F1FB72B031300346E300C1E1F
:1027C000DF2B99002C300C1EE32B99000A3084007B
:1027D00003171108B9001008B800031364232C3044
:1027E0000C1EF02B99000A30840003171308B9005F
:1027F0001208B800031364232C300C1EFD2B990023
:102800000A30840003171508B9001408B800031330
:1028100064232C300C1E0A2C99000A308400031704
:102820001708B9001608B800031364232C300C1ED7
:10283000172C99000A30840003171908B9001808EA
:10284000B800031364232C300C1E242C99000A308A
:10285000840003171B08B9001A08B8000313642387
:102860002C300C1E312C99000A30840003172308E9
:10287000B9002208B800031364232C300C1E3E2C30
:1028800099000A30840003172508B9002408B8000D
:10289000031364232C300C1E4B2C99000A30840047
:1028A00003172108B9002008B800031364232C3053
:1028B0000C1E582C99000A30840003172708B90011
:1028C0002608B800031364230D300C1E652C9900F4
:1028D0000A300C1E692C99008A150A160B2D6F30D0
:1028E0000C1E702C99002C300C1E742C99000A3090
:1028F00084004B080317B90003134A080317B800F4
:10290000031364232C300C1E832C99000A3084009E
:102910004D080317B90003134C080317B80003133D
:1029200064232C300C1E922C99000A3084004F082E
:102930000317B90003134E080317B80003136423E9
:102940002C300C1EA12C99000A308400510803176A
:10295000B900031350080317B800031364232C3085
:102960000C1EB02C99000A30840053080317B900DC
:10297000031352080317B800031364232C300C1EF2
:10298000BF2C99000A30840055080317B9000313BF
:1029900054080317B800031364232C300C1ECE2CEC
:1029A00099000A3084005D080317B90003135C081E
:1029B0000317B800031364232C300C1EDD2C990080
:1029C0000A3084005F080317B90003135E08031779
:1029D000B800031364232C300C1EEC2C99000A3031
:1029E00084005B080317B90003135A080317B800E3
:1029F000031364232C300C1EFB2C99000A30840036
:102A000061080317B900031360080317B800031324
:102A100064230D300C1E0A2D99000A300C1E0E2D59
:102A200099008A150A160B2D831603171408403CCB
:102A300003181F2D413014020A3E9500222D30301C
:102A4000140295001508F800831203130034780867
:102A500003173D08BF006430C0000A120313372576
:102A60000A1677080317BD0078083030031D3F2D84
:102A7000BE1C492DBE19492D3E1A2030422DBE11D3
:102A80003E123E14F807780803130C1E452D9900DA
:102A900003173D08BF000A30C0000A120313372590
:102AA0000A1677080317BD0078083030031D5E2D25
:102AB000BE19652D3E1C652D3E1A2030F80778089A
:102AC00003130C1E612D990003173030BD073D081C
:102AD00003130C1E692D990000340317B801B901C6
:102AE000BA01BC0183160313220803179400831252
:102AF0000313142578080317B800380EBD00F03012
:102B0000BD058316031323080317940083120313D0
:102B10001425780803173D07B8008316031325080A
:102B20000317940083120313142578080317B900C0
:102B3000390EBD00F030BD058316031326080317B8
:102B40009400831203131425780803173D07B90076
:102B50008316031328080317940083120313142504
:102B600078080317BA003A0EBD00F030BD05831691
:102B700003132908031794008312031314257808FC
:102B800003173D07BA008316031311141118C62D3D
:102B90008312031738088316910083120313FF2151
:102BA000031739088316910083120313FF2183163C
:102BB00091149118D92D0130831203173807BD00E5
:102BC0008316910083120313FF2172300C1EE62D31
:102BD000990003173A08013C0318062E0130F7004C
:102BE0000A120313EF270A1678080317BB002C30CC
:102BF00003130C1EF92D990003173B08BD00033089
:102C0000BE00031327250317BA03EA2DF7010A12A2
:102C10000313EF270A1678080317BB002C300313A1
:102C20000C1E102E990003173B08BD000330BE0098
:102C3000031327258316111511191C2E0D3083122D
:102C40000C1E202E99000A300C1E242E99008A1585
:102C50000A160B2D74300C1E2B2E99002C300C1ED6
:102C60002F2E99003D080317BD000330BE0003134B
:102C700027252C300C1E3A2E99003E080317BD0064
:102C80000330BE00031327250D300C1E452E99007E
:102C90000A300C1E492E99008A150A160B2D023097
:102CA0000317BD00BE01A0303D0784008313000858
:102CB0002C3C0319862EA0303D07840083130008A6
:102CC0000A3C0319862EA0303D07840083130008B8
:102CD0000D3C0319862E38303E07F8000130FA000B
:102CE0000318FA0A7808BF007A08C000A0303D0730
:102CF000840083130008C1003F0884008313401838
:102D0000831741088000BD0ABE0A532E38303E07A3
:102D10008400831780010130C1003830C0000A12DE
:102D20008A150313C4250A168A117808C100A03039
:102D300003173D078400831300080A3C0319A82EDB
:102D4000A0303D078400831300080D3C031DBB2EFB
:102D5000BF013F080A120313C5200A160317BF0A52
:102D6000F70003130C1EB22E9900143003173F0214
:102D7000031DA92E192FBD0ABE01A0303D078400F6
:102D8000831300080A3C0319E82EA0303D07840095
:102D9000831300080D3C0319E82E38303E07F80075
:102DA0000130FA000318FA0A7808BF007A08C00058
:102DB000A0303D07840083130008C1003F08840051
:102DC00083134018831741088000BD0ABE0ABD2E38
:102DD00038303E078400831780010130C10038304D
:102DE000C0000A128A150313C4250A168A1178082E
:102DF000C000C21476300C1EFB2E99000D300C1E44
:102E0000FF2E99000A300C1E032F99004218062F3E
:102E100091010830F80005389200D73083169200EF
:102E20008312BF012D130B1283160C108C14831206
:102E3000031703138A150A160B2D0317B8018316FF
:102E40000313220803179400831203131425780830
:102E50000317B800380EB900F030B9058316031314
:102E6000230803179400831203131425780803170B
:102E70003907B80083160313111411183D2F83125C
:102E8000031738088316910083120313FF2183165A
:102E900025080317940083120313142578080317D9
:102EA000B800380EB900F030B905831603132608B0
:102EB00003179400831203131425780803173907A6
:102EC000B80038088316910083120313FF2183167C
:102ED0002808031794008312031314257808031796
:102EE000B800380EB900F030B9058316031329086D
:102EF0000317940083120313142578080317390766
:102F0000B80038088316910083120313FF2183163B
:102F100011151119892F773083120C1E8D2F9900EE
:102F20000D300C1E912F99000A300C1E952F990020
:102F30008A150A160B2D7A300C1E9C2F99000D3025
:102F40000C1EA02F99000A300C1EA42F99008A0194
:102F500000288A150A160B2D0317B80138080A1223
:102F60000313C5200A160317B80AF70003130C1E33
:102F7000B72F9900143003173802031DAE2F031327
:062F80008A150A160B2D54
:103000000317B801B901EC01831603132208031753
:1030100094008A118312031314258A157808031764
:10302000B800380E83169000F03090050313230883
:10303000031794008A118312031314258A15780844
:103040008316031710078312B8008316031325088D
:10305000031794008A118312031314258A15780824
:103060000317B900390E83169000F0309005031352
:103070002608031794008A118312031314258A1556
:1030800078088316031710078312B90083160313F9
:103090002808031794008A118312031314258A1534
:1030A00078080317EC006C0E83169000F030900542
:1030B00003132908031794008A118312031314259C
:1030C0008A1578088316031710078312EC00ED01A8
:1030D0006C086D020318C0283A306D078316900003
:1030E000013091000318910A0B3083126D076D07B0
:1030F0006D07A03E8400831300088316920094009D
:103100008A118312031314258A15831603171008D6
:103110008400831311188317780880003A308312D3
:103120006D0783169000013091000318910A3A3020
:1031300083126D0784008317000E83169200F0300F
:1031400092050C3083126D076D076D07A03E840059
:10315000831300088316930094008A1183120313CB
:1031600014258A157808831603179207100884001F
:10317000831311188317120880008312ED0A682840
:103180008316031311141118C32883120317380868
:10319000831691008A1183120313FF218A150317E6
:1031A0003908831691008A1183120313FF218A15AF
:1031B0000317ED016C086D020318EE283A306D0715
:1031C0008400831700088316900091008A118312EF
:1031D0000313FF218A150317ED0ADA288316031358
:1031E00011151119F128793083120C1EF528990058
:1031F0000D300C1EF92899000A300C1EFD2899008C
:103200008A150A160B2D831621082C3C0319152943
:1032100021080A3C0319152921080D3C0319152919
:103220008312AE012D120B2D83162008413A831212
:1032300003195429033A03195829013A03195C293F
:10324000073A0319F129013A0319F529033A031939
:10325000F929013A0319AF2A0F3A0319C02A013A92
:103260000319C42A033A0319DE2A063A0319E22A8B
:10327000023A0319E62A013A0319EA2A1D3A031908
:10328000EE2A063A0319F22A023A0319F62A013AFB
:103290000319FA2A0F3A0319FE2A013A0319012DDC
:1032A000033A0319032D072D8A1100288A150B2DC7
:1032B0000A12C62E0A160B2DAE012D120130F60091
:1032C00002300317B900FA30E8000A128A1103131A
:1032D000DB270A168A150317B90B63292B30031352
:1032E0000C1E702999002B300C1E742999002B306C
:1032F0000C1E7829990004300317B900C830E80083
:103300000A128A110313DB270A168A150317B90B51
:103310007E290313AE012D120317B90139080A12D1
:103320008A110313DE200A168A150317B90AF7005B
:1033300003130C1E99299900043003173902031D49
:103340008E290630B900FA30E8000A128A110313F8
:10335000DB270A168A150317B90BA3298316031353
:10336000560883120317B8000313AE010317B901FF
:1033700039080A128A110313E7200A168A1503175F
:10338000B90AF70003130C1EC3299900093003176B
:103390003902031DB8290430B900FA30E8000A12D6
:1033A0008A110313DB270A168A150317B90BCD29D7
:1033B000F601633003130C1EDB2999002C300C1E20
:1033C000DF2999000317380803130C1EE52999001B
:1033D0000D300C1EE92999000A300C1EED299900C8
:1033E0000B2D0A12F92E0A160B2D0A12D02F0A16CF
:1033F0000B2D66300C1EFA2999002C300C1EFE296C
:1034000099004130840046080317BB0003134508A8
:103410000317BA00031344080317B9000313430842
:103420000317B8000408BC00BB1F232ABC03BC164A
:10343000B809B909BA09BB09B80A0319B90A0319C5
:10344000BA0A0319BB0A3B30C3009A30C200CA3023
:10345000C100C0010A30BE003B08C7003A08C600E0
:103460003908C5003808C4004308CB004208CA0028
:103470004108C9004008C8008A1103133F218A157A
:1034800000080317B800840A0008B900840A00087D
:10349000BA00840A0008BB00F708031D622A3E0830
:1034A000013A0319622A3C080319642A0F393E02C3
:1034B00003195C2A0318892ABC1B892A3C1B642A2D
:1034C0002030822A2030BC05BC1E722ABC1277082C
:1034D000BC002D3003130C1E6B2A990003173C0807
:1034E000F700BC013030BC1E822ABC127708BC0039
:1034F0002D3003130C1E7A2A990003173C08F7009D
:10350000BC013030F707770803130C1E852A990099
:1035100003174308C7004208C6004108C500400819
:10352000C400CB01CA01C9010A30C8008A110313C3
:103530003F218A157A080317C3007908C20078086A
:10354000C1007708C000BE0B2C2A0D3003130C1EDF
:10355000A72A99000A300C1EAB2A99000B2DC60130
:10356000C501C401C30167300C1EB42A99000D3097
:103570000C1EB82A99000A300C1EBC2A99000B2D8B
:103580008A1183298A150B2D69300C1EC52A9900D2
:103590002C300C1EC92A990070080317BB00573045
:1035A000BC008A110313D8218A150D300C1ED62AAF
:1035B00099000A300C1EDA2A99000B2D8A11132A61
:1035C0008A150B2D8A11902A8A150B2D8A11DE2B54
:1035D0008A150B2D8A116F2C8A150B2D8A116D2DD2
:1035E0008A150B2D8A112A2E8A150B2D8A114F2E22
:1035F0008A150B2D8A111D2F8A150B2D0317100804
:10360000B800B9011108BA00BB01BB011208BC0027
:10361000BD011308BE00BF01BF01783003130C1EAB
:103620000F2B99000317380803130C1E152B990054
:1036300003173A0803130C1E1B2B990003173C08B1
:1036400003130C1E212B990003173E0803130C1EB5
:10365000272B990003171408B800B9011508BA0000
:10366000BB01BB011608BC00BD011708BE00BF01AD
:10367000BF01140803130C1E3B2B990003173A08D3
:1036800003130C1E412B990003173C0803130C1E57
:10369000472B990003173E0803130C1E4D2B99006E
:1036A00003171808B800B9011908BA00BB01BB011B
:1036B0001A08BC00BD011B08BE00BF01BF011808ED
:1036C00003130C1E612B990003173A0803130C1EF9
:1036D000672B990003173C0803130C1E6D2B9900F0
:1036E00003173E0803130C1E732B990003172208BF
:1036F000B800B9012308BA00BB01BB012408BC0013
:10370000BD012508BE00BF01BF01220803130C1E26
:10371000872B990003173A0803130C1E8D2B990071
:1037200003173C0803130C1E932B990003173E0844
:1037300003130C1E992B990003172008B800B90138
:103740002108BA00BB01BB012608BC00BD01270847
:10375000BE00BF01BF01200803130C1EAD2B990052
:1037600003173A0803130C1EB32B990003173C08E8
:1037700003130C1EB92B990003173E0803130C1EEC
:10378000BF2B99004A080317B800B90103134B086F
:103790000317BA00BB01BB0103134C080317BC009D
:1037A000BD0103134D080317BE00BF01BF01380858
:1037B00003130C1ED92B990003173A0803130C1E90
:1037C000DF2B990003173C0803130C1EE52B99000F
:1037D00003173E0803130C1EEB2B99004E0803172A
:1037E000B800B90103134F080317BA00BB01BB01AE
:1037F000031350080317BC00BD010313510803173E
:10380000BE00BF01BF01380803130C1E052C990030
:1038100003173A0803130C1E0B2C990003173C08DE
:1038200003130C1E112C990003173E0803130C1EE2
:10383000172C990052080317B800B9010313530855
:103840000317BA00BB01BB01031354080317BC00E4
:10385000BD01031355080317BE00BF01BF0138089F
:1038600003130C1E312C990003173A0803130C1E86
:10387000372C990003173C0803130C1E3D2C9900AC
:1038800003173E0803130C1E432C99005C08031712
:10389000B800B90103135D080317BA00BB01BB01EF
:1038A00003135E080317BC00BD0103135F08031771
:1038B000BE00BF01BF01380803130C1E5D2C990028
:1038C00003173A0803130C1E632C990003173C08D6
:1038D00003130C1E692C990003173E0803130C1EDA
:1038E0006F2C99005A080317B800B90103135B083D
:1038F0000317BA00BB01BB01031360080317BC0028
:10390000BD01031361080317BE00BF01BF013808E2
:1039100003130C1E892C990003173A0803130C1E7D
:103920008F2C990003173C0803130C1E952C99004B
:1039300003173E0803130C1E9B2C99004308031722
:10394000B800B901BA01BB01031344080317BD0055
:10395000031345080317BE00031346080317BF00EF
:10396000C001BE01BF01C001031345080317C20017
:10397000031346080317C300C401C501C301C401F2
:10398000C501031346080317C700C801C901CA01CE
:10399000C801C901CA0103132A080C1ECD2C9900C5
:1039A0002B080C1ED12C990070080C1ED52C9900E8
:1039B0003D080C1ED92C99003E080C1EDD2C9900E8
:1039C0000317380803130C1EE32C990003173D0856
:1039D00003130C1EE92C99000317420803130C1E55
:1039E000EF2C99000317470803130C1EF52C9900C0
:1039F0000D300C1EF92C99000A300C1EFD2C99007C
:103A00000B2D00280B2D8A119B2F8A150B2D8A1147
:103A1000AC2F8A150B2DAE012D128A150A169D2D7D
:103A2000840183131F308305713083168F000F08C4
:103A30000317871522300313990000309A00A6302F
:103A40009800903083129800A915290883168700E2
:103A50008312291629088316870013309300293012
:103A600083129400831694171413FF3093002830A8
:103A700083129400831603170908C03989000313C1
:103A80001F129F12003003178800831287018801DC
:103A90008901FF300313A900AA01AB01AC012D1469
:103AA000AD142D15AD152D12AE01AD12BD01BE0127
:103AB000BF012D13C001C101AD134210C21042114C
:103AC000C301C401C501C601C701C801C901E201A2
:103AD000E301C2111030F100F201F301F401F5012C
:103AE000F601FC01FD0102300317AC000330AD000C
:103AF000FC30AE00FD30AF00FE30B0000230B1004F
:103B0000FE30B200FD30B300FB30B4000330B5002E
:103B10000230B600B700031342120A128A11C32DF5
:103B20000A168A15F0080319982D0A1229290A166F
:0E3B30002D1E9D2D2D1D9D2D0329982D63000A
:04400E00E52FFF3E5D
:00000001FF
